:020000040000FA
:0200000032D0FC
:0200080025D001
:08001800D8CF01F0E8CF00F0A1
:10002000E0CF02F0EACF03F0E9CF04F09EAA02D0BD
:100030009DBA6DD39EA802D09DB862D3FF0004C0C4
:10004000E9FF03C0EAFF02C0E0FF00C0E8FF01C013
:10005000D8FF1000EACF05F0E9CF06F0A1A202D048
:10006000A0B227D0FF00896A8A6A8B6A926A936A73
:10007000800E946E070EC16EC26A096A0A6A0B6A24
:10008000100E0C6E080EC1EC04F0080EDEEC04F04D
:10009000F40EF26FF36F00EE00F010EE00F055DB9F
:1000A00003D854EC04F0FDD7010EB16EA282A082F9
:1000B0001200A192500EB26EB3680950896E0A50B8
:1000C0008A6E0B508B6EF251F35D14E0F2C0E9FFC3
:1000D000EA6A030EF22702E1F40EF26FEF5000EC31
:1000E00003F0EE50E826200FE16EE26AEE50E66E75
:1000F000EE50E66E210604E2200602E22168099431
:10010000230604E2220602E223680992250604E29D
:10011000240602E225680990270604E2260602E288
:1001200027680996290604E2280602E22968099848
:100130002B0604E22A0602E22B68099A2D0604E245
:100140002C0602E22D680A9E2F0604E22E0602E229
:100150002F680A9C310604E2300602E231680A9AEE
:10016000330604E2320602E233680A98350604E2F6
:10017000340602E235680A96370604E2360602E2E1
:1001800037680A94390604E2380602E239680A92AE
:100190003B0604E23A0602E23B680A903D0604E2AE
:1001A0003C0602E23D680B9A3F0604E23E0602E28C
:1001B0003F680B98C5D2535026E0535024E00F0EF1
:1001C000F76E52C0F6FF0800F5501CE0F504086E0B
:1001D000EA6AF3C0E9FF0850EE6E53505324F66EFE
:1001E00008500C24F76E0900F5CF07F00900F55010
:1001F000EE6E0750EE6EE95002E0F36F1200F40E5F
:10020000F36F12001200120012007B0E525C01E02C
:100210001200096A0A6A0B6A896A8A6A8B6A120082
:10022000525016EC01F00C6E00001200800FE84AEC
:10023000700CE84A600CE84A500CE84A400CE84A66
:10024000300CE84A200C100CF66E0F0EF76E08000A
:10025000F55012001200030E146EF80E156E120007
:1002600014C0EAFF15C0E9FFEE6EEACF14F0E9CF43
:1002700015F0EA50030807E0EA50040804E0EA50E9
:10028000050801E0E8D712001450050849E11550AF
:10029000000846E103EEF8F0EE507D0841E1EE5033
:1002A00073083EE1EE506E083BE1EE50610838E124
:1002B000EE50720835E1EE50060832E10000EE50D3
:1002C00016EC01F0106E10082BE0EE5024EC01F05B
:1002D00027E0E8061026800E0D6ED890EE32D8B0DA
:1002E000EF8EED52EECF08F0ED50EE6E08C0EEFF4F
:1002F000040E126E000E0F6E0D2EEFD7096A0A6AF9
:100300000B6A896A8A6A8B6A91EC01F0096A0A6A47
:100310000B6A896A8A6A8B6A020EDEEC04F01200AC
:100320001200000E136E000E116EA7EC01F0400ECD
:10033000116E136EA7EC01F0800E116E136EA7EC18
:1003400001F0C00E116E136EA7EC01F012000F50F9
:10035000F86E1050F76E1150F66EA68EA69CA6840D
:10036000A688F29E550EA76EAA0EA76EA682F28EE2
:100370000A00080E0E6E1250EA6E1350E96E080E57
:100380000D6EEE50F56E0F000D2EFBD7A68EA69CBF
:10039000A684F29E550EA76EAA0EA76EA682F28EB6
:1003A0000E2EEDD7A6940F50F86E1050F76E115028
:1003B000F66E1250EA6E1350E96E400E0D6E090093
:1003C000F550EE5E03E10D2EFAD71200100EC1ECCF
:0403D00004F0FCD762
:10060000040DF950F350F9260984120009821200F2
:10061000098012000986120009881200098A120056
:100620000A8E12000A8C12000A8A12000A8812002E
:100630000A8612000A8412000A8212000A8012003E
:080640000B8A12000B88120066
:1007000056A202D09D989BD488D8AD6E98D4ABB237
:1007100007D0ABB40AD056B40ED0AE5061D88FD447
:10072000AB98AB88FA0E3CD88AD4AE50AB98AB8865
:10073000FC0E36D884D4AE500B80FB0E31D87FD45B
:1007400006C0E9FF05C0EAFF1100C00E94124F0E6B
:10075000AF6E240EAC6E900EAB6E566A516A526A42
:10076000536A506A546A556A09D811D89D8A9D887F
:100770009F9A9F98D08EF28CF28E1200000E5A6EC5
:100780005C6E620E5B6E5D6E569056821200000EBD
:100790005E6E606E720E5F6E616E569456861200CB
:1007A0009D9856B01BD05CC0EAFF5DC0E9FFEE6EBD
:1007B000000EEA6205D0720EE96202D000EE62F02D
:1007C000EACF5CF0E9CF5DF05A505C6204D05B5038
:1007D0005D6201D0568056929D8812009D8812005D
:1007E00056B41AD060C0EAFF61C0E9FFEE6E000E99
:1007F000EA6205D0820EE96202D000EE72F0EACF22
:1008000060F0E9CF61F05E50606204D05F506162D9
:1008100001D0568456961200120056B21CD05AC00F
:10082000EAFF5BC0E9FFEECF59F0000EEA6205D0A7
:10083000720EE96202D000EE62F0EACF5AF0E9CF20
:100840005BF05C505A6204D05D505B6201D056820E
:10085000569059501200000C9D9A56B61DD05EC09D
:10086000EAFF5FC0E9FFEECF58F0000EEA6205D064
:10087000820EE96202D000EE72F0EACF5EF0E9CFBC
:100880005FF060505E6204D061505F6201D05686B6
:10089000569458509D8A12009D8A000C56B612003C
:1008A000DBDF7EDFFBD7120056B61200D5DF506EBD
:1008B000505050AE35D0516E51AC2ED05150F00B3F
:1008C000E0082AE05150F00BF00822E15150F20804
:1008D00023E05150F1081CE05150F30819E0515049
:1008E000F00844E05150E84AB5D4E84AB3D4E84AA5
:1008F000B1D4E84AAFD4E84AADD4E84AABD4E84A28
:10090000A9D4E84AA7D4E84ABFD4E84AA3D412003D
:10091000546A010E556E1200546A020E556E120092
:1009200055BE9ED454660FD050C052F0542A545035
:10093000555C01E01200546AD60E515C20E0C60EF0
:10094000515C1BE0120050C053F0546A960E515C8B
:1009500010E0860E515C0FE0B60E515C0DE0A60E65
:10096000515C0CE0E60E515C0BE01200800E556EFF
:1009700072D4DBEF00F047D448D452D46BD46AD49D
:1009800069D4506E516A526A5050536E515052643D
:100990008B8052608B90000000000000000000007F
:1009A00000000000523EF2D7532EF0D7513EECD754
:1009B0008B80516A526A536A506A1200506E516AB3
:1009C000526A5050536E515052648B9052608B80DB
:1009D0000000000000000000000000000000523E87
:1009E000F2D7532EF0D7513EECD78B90516A526A12
:0609F000536A506A120078
:100F000000000000000000000000000000000000E1
:100F100000000000000000000000000000000000D1
:100F200000000000000000000000000000000000C1
:100F30000000000000000000000000000809070A8F
:100F4000060B050C040D0302010E0F10000000003B
:100F50000000000000000000000000000000000091
:100F60000000000000000000000000000000000081
:100F70000000000000000000000000000000000071
:1010000000002100230024002500270028002900DB
:101010002B002C002D002F00300031003300340055
:101020003600370038003A003B003C003E003F00ED
:1010300040004200430044004600470048004A0088
:101040004B004C004E004F00500052005300540023
:101050005600570058005A005B005C005E005F00BD
:1010600060006200630065006600670069006A0056
:101070006B006D006E006F007100720073007500F0
:101080007600770079007A007B007D007E007F008B
:1010900081008200830085008600870089008A0025
:1010A0008C008D008E0090009100920094009500BD
:1010B0009600980099009A009C009D009E00A00058
:1010C000A100A200A400A500A600A800A900AA00F3
:1010D000AC00AD00AE00B000B100B200B400B5008D
:1010E000B600B800B900BB00BC00BD00BF00C00026
:1010F000C100C300C400C500C700C800C900CB00C0
:1011000000002100230024002500270028002900DA
:101110002B002C002D002F00300031003300340054
:101120003600370038003A003B003C003E003F00EC
:1011300040004200430044004600470048004A0087
:101140004B004C004E004F00500052005300540022
:101150005600570058005A005B005C005E005F00BC
:1011600060006200630065006600670069006A0055
:101170006B006D006E006F007100720073007500EF
:101180007600770079007A007B007D007E007F008A
:1011900081008200830085008600870089008A0024
:1011A0008C008D008E0090009100920094009500BC
:1011B0009600980099009A009C009D009E00A00057
:1011C000A100A200A400A500A600A800A900AA00F2
:1011D000AC00AD00AE00B000B100B200B400B5008C
:1011E000B600B800B900BB00BC00BD00BF00C00025
:1011F000C100C300C400C500C700C800C900CB00BF
:1012000000002100230024002500270028002900D9
:101210002B002C002D002F00300031003300340053
:101220003600370038003A003B003C003E003F00EB
:1012300040004200430044004600470048004A0086
:101240004B004C004E004F00500052005300540021
:101250005600570058005A005B005C005E005F00BB
:1012600060006200630065006600670069006A0054
:101270006B006D006E006F007100720073007500EE
:101280007600770079007A007B007D007E007F0089
:1012900081008200830085008600870089008A0023
:1012A0008C008D008E0090009100920094009500BB
:1012B0009600980099009A009C009D009E00A00056
:1012C000A100A200A400A500A600A800A900AA00F1
:1012D000AC00AD00AE00B000B100B200B400B5008B
:1012E000B600B800B900BB00BC00BD00BF00C00024
:1012F000C100C300C400C500C700C800C900CB00BE
:1013000000002100230024002500270028002900D8
:101310002B002C002D002F00300031003300340052
:101320003600370038003A003B003C003E003F00EA
:1013300040004200430044004600470048004A0085
:101340004B004C004E004F00500052005300540020
:101350005600570058005A005B005C005E005F00BA
:1013600060006200630065006600670069006A0053
:101370006B006D006E006F007100720073007500ED
:101380007600770079007A007B007D007E007F0088
:1013900081008200830085008600870089008A0022
:1013A0008C008D008E0090009100920094009500BA
:1013B0009600980099009A009C009D009E00A00055
:1013C000A100A200A400A500A600A800A900AA00F0
:1013D000AC00AD00AE00B000B100B200B400B5008A
:1013E000B600B800B900BB00BC00BD00BF00C00023
:1013F000C100C300C400C500C700C800C900CB00BD
:1014000000002100230024002500270028002900D7
:101410002B002C002D002F00300031003300340051
:101420003600370038003A003B003C003E003F00E9
:1014300040004200430044004600470048004A0084
:101440004B004C004E004F0050005200530054001F
:101450005600570058005A005B005C005E005F00B9
:1014600060006200630065006600670069006A0052
:101470006B006D006E006F007100720073007500EC
:101480007600770079007A007B007D007E007F0087
:1014900081008200830085008600870089008A0021
:1014A0008C008D008E0090009100920094009500B9
:1014B0009600980099009A009C009D009E00A00054
:1014C000A100A200A400A500A600A800A900AA00EF
:1014D000AC00AD00AE00B000B100B200B400B50089
:1014E000B600B800B900BB00BC00BD00BF00C00022
:1014F000C100C300C400C500C700C800C900CB00BC
:1015000000002100230024002500270028002900D6
:101510002B002C002D002F00300031003300340050
:101520003600370038003A003B003C003E003F00E8
:1015300040004200430044004600470048004A0083
:101540004B004C004E004F0050005200530054001E
:101550005600570058005A005B005C005E005F00B8
:1015600060006200630065006600670069006A0051
:101570006B006D006E006F007100720073007500EB
:101580007600770079007A007B007D007E007F0086
:1015900081008200830085008600870089008A0020
:1015A0008C008D008E0090009100920094009500B8
:1015B0009600980099009A009C009D009E00A00053
:1015C000A100A200A400A500A600A800A900AA00EE
:1015D000AC00AD00AE00B000B100B200B400B50088
:1015E000B600B800B900BB00BC00BD00BF00C00021
:1015F000C100C300C400C500C700C800C900CB00BB
:1016000000002100230024002500270028002900D5
:101610002B002C002D002F0030003100330034004F
:101620003600370038003A003B003C003E003F00E7
:1016300040004200430044004600470048004A0082
:101640004B004C004E004F0050005200530054001D
:101650005600570058005A005B005C005E005F00B7
:1016600060006200630065006600670069006A0050
:101670006B006D006E006F007100720073007500EA
:101680007600770079007A007B007D007E007F0085
:1016900081008200830085008600870089008A001F
:1016A0008C008D008E0090009100920094009500B7
:1016B0009600980099009A009C009D009E00A00052
:1016C000A100A200A400A500A600A800A900AA00ED
:1016D000AC00AD00AE00B000B100B200B400B50087
:1016E000B600B800B900BB00BC00BD00BF00C00020
:1016F000C100C300C400C500C700C800C900CB00BA
:1017000000002100230024002500270028002900D4
:101710002B002C002D002F0030003100330034004E
:101720003600370038003A003B003C003E003F00E6
:1017300040004200430044004600470048004A0081
:101740004B004C004E004F0050005200530054001C
:101750005600570058005A005B005C005E005F00B6
:1017600060006200630065006600670069006A004F
:101770006B006D006E006F007100720073007500E9
:101780007600770079007A007B007D007E007F0084
:1017900081008200830085008600870089008A001E
:1017A0008C008D008E0090009100920094009500B6
:1017B0009600980099009A009C009D009E00A00051
:1017C000A100A200A400A500A600A800A900AA00EC
:1017D000AC00AD00AE00B000B100B200B400B50086
:1017E000B600B800B900BB00BC00BD00BF00C0001F
:1017F000C100C300C400C500C700C800C900CB00B9
:1018000000002100230024002500270028002900D3
:101810002B002C002D002F0030003100330034004D
:101820003600370038003A003B003C003E003F00E5
:1018300040004200430044004600470048004A0080
:101840004B004C004E004F0050005200530054001B
:101850005600570058005A005B005C005E005F00B5
:1018600060006200630065006600670069006A004E
:101870006B006D006E006F007100720073007500E8
:101880007600770079007A007B007D007E007F0083
:1018900081008200830085008600870089008A001D
:1018A0008C008D008E0090009100920094009500B5
:1018B0009600980099009A009C009D009E00A00050
:1018C000A100A200A400A500A600A800A900AA00EB
:1018D000AC00AD00AE00B000B100B200B400B50085
:1018E000B600B800B900BB00BC00BD00BF00C0001E
:1018F000C100C300C400C500C700C800C900CB00B8
:1019000000002100230024002500270028002900D2
:101910002B002C002D002F0030003100330034004C
:101920003600370038003A003B003C003E003F00E4
:1019300040004200430044004600470048004A007F
:101940004B004C004E004F0050005200530054001A
:101950005600570058005A005B005C005E005F00B4
:1019600060006200630065006600670069006A004D
:101970006B006D006E006F007100720073007500E7
:101980007600770079007A007B007D007E007F0082
:1019900081008200830085008600870089008A001C
:1019A0008C008D008E0090009100920094009500B4
:1019B0009600980099009A009C009D009E00A0004F
:1019C000A100A200A400A500A600A800A900AA00EA
:1019D000AC00AD00AE00B000B100B200B400B50084
:1019E000B600B800B900BB00BC00BD00BF00C0001D
:1019F000C100C300C400C500C700C800C900CB00B7
:101A000000002100230024002500270028002900D1
:101A10002B002C002D002F0030003100330034004B
:101A20003600370038003A003B003C003E003F00E3
:101A300040004200430044004600470048004A007E
:101A40004B004C004E004F00500052005300540019
:101A50005600570058005A005B005C005E005F00B3
:101A600060006200630065006600670069006A004C
:101A70006B006D006E006F007100720073007500E6
:101A80007600770079007A007B007D007E007F0081
:101A900081008200830085008600870089008A001B
:101AA0008C008D008E0090009100920094009500B3
:101AB0009600980099009A009C009D009E00A0004E
:101AC000A100A200A400A500A600A800A900AA00E9
:101AD000AC00AD00AE00B000B100B200B400B50083
:101AE000B600B800B900BB00BC00BD00BF00C0001C
:101AF000C100C300C400C500C700C800C900CB00B6
:101B000000002100230024002500270028002900D0
:101B10002B002C002D002F0030003100330034004A
:101B20003600370038003A003B003C003E003F00E2
:101B300040004200430044004600470048004A007D
:101B40004B004C004E004F00500052005300540018
:101B50005600570058005A005B005C005E005F00B2
:101B600060006200630065006600670069006A004B
:101B70006B006D006E006F007100720073007500E5
:101B80007600770079007A007B007D007E007F0080
:101B900081008200830085008600870089008A001A
:101BA0008C008D008E0090009100920094009500B2
:101BB0009600980099009A009C009D009E00A0004D
:101BC000A100A200A400A500A600A800A900AA00E8
:101BD000AC00AD00AE00B000B100B200B400B50082
:101BE000B600B800B900BB00BC00BD00BF00C0001B
:101BF000C100C300C400C500C700C800C900CB00B5
:101C000000002100230024002500270028002900CF
:101C10002B002C002D002F00300031003300340049
:101C20003600370038003A003B003C003E003F00E1
:101C300040004200430044004600470048004A007C
:101C40004B004C004E004F00500052005300540017
:101C50005600570058005A005B005C005E005F00B1
:101C600060006200630065006600670069006A004A
:101C70006B006D006E006F007100720073007500E4
:101C80007600770079007A007B007D007E007F007F
:101C900081008200830085008600870089008A0019
:101CA0008C008D008E0090009100920094009500B1
:101CB0009600980099009A009C009D009E00A0004C
:101CC000A100A200A400A500A600A800A900AA00E7
:101CD000AC00AD00AE00B000B100B200B400B50081
:101CE000B600B800B900BB00BC00BD00BF00C0001A
:101CF000C100C300C400C500C700C800C900CB00B4
:101D00000000D700DE00E500EB00F200F900000162
:101D100007010E0115011C012201290130013701C3
:101D20003E0145014C0152015901600167016E01FC
:101D300075017C0183018901900197019E01A50134
:101D4000AC01B301B901C001C701CE01D501DC016D
:101D5000E301EA01F001F701FE0105020C021302A2
:101D60001A02200227022E0235023C0243024A02D6
:101D7000510257025E0265026C0273027A0281020E
:101D800088028E0295029C02A302AA02B102B80246
:101D9000BE02C502CC02D302DA02E102E802EF027F
:101DA000F502FC0203030A03110318031F032503B2
:101DB0002C0333033A03410348034F0356035C03E8
:101DC00063036A03710378037F0386038C03930321
:101DD0009A03A103A803AF03B603BD03C303CA0359
:101DE000D103D803DF03E603ED03F303FA03010491
:101DF00008040F0416041D0424042A0431043804C2
:101E00000000D700DE00E500EB00F200F900000161
:101E100007010E0115011C012201290130013701C2
:101E20003E0145014C0152015901600167016E01FB
:101E300075017C0183018901900197019E01A50133
:101E4000AC01B301B901C001C701CE01D501DC016C
:101E5000E301EA01F001F701FE0105020C021302A1
:101E60001A02200227022E0235023C0243024A02D5
:101E7000510257025E0265026C0273027A0281020D
:101E800088028E0295029C02A302AA02B102B80245
:101E9000BE02C502CC02D302DA02E102E802EF027E
:101EA000F502FC0203030A03110318031F032503B1
:101EB0002C0333033A03410348034F0356035C03E7
:101EC00063036A03710378037F0386038C03930320
:101ED0009A03A103A803AF03B603BD03C303CA0358
:101EE000D103D803DF03E603ED03F303FA03010490
:101EF00008040F0416041D0424042A0431043804C1
:101F0000000060007F009E00BE00DE00FD001C019E
:101F10003C015C017B019A01BA01DA01F901180266
:101F20003802580277029602B602D602F50214036E
:101F30003403540373039203B203D203F103100476
:101F4000300450046F048E04AE04CE04ED040C057E
:101F50002C054C056B058A05AA05CA05E905080686
:101F60002806480667068606A606C606E50604078E
:101F70002407440763078207A207C207E107000896
:101F8000200840085F087E089E08BE08DD08FC089F
:101F90001C093C095B097A099A09BA09D909F809A7
:101FA000180A380A570A760A960AB60AD50AF40AAF
:101FB000140B340B530B720B920BB20BD10BF00BB7
:101FC000100C300C4F0C6E0C8E0CAE0CCD0CEC0CBF
:101FD0000C0D2C0D4B0D6A0D8A0DAA0DC90DE80DC7
:101FE000080E280E470E660E860EA60EC50EE40ECF
:101FF000040F240F430F620F820FA20FC10FE00FD7
:020000040030CA
:03000100260A00CC
:02000500018177
:060008000FC00FE00F40E5
:00000001FF
